:020000040000FA
:060000004BEF1DF01200A1
:020006001200E6
:0600080023EF1BF01200C3
:02000E000100EF
:0C001000C43A0000D70000000900000006
:04001C00D9CFE6FF53
:10002000E1CFD9FF81E941E8240EAC6E900EAB6EB2
:10003000B896150EAF6E93928192016AD8900150D6
:1000400002E6320E015C02E2012AF8D78182000149
:10005000140ED96FD95101E0FDD7AE50016EAE50EC
:10006000016E016AD890015002E6050E015C0CE2B7
:10007000550EE66E54EC0AF041E961EC0AF0000915
:1000800001E102D0012AEED70001EA69E96B42E9F9
:10009000E7CFD9FF1200D9CFE6FFE1CFD9FF81E941
:1000A00045E8E66AE66AE66AE66AE1EC09F044E9F0
:1000B0000001E06FE03502E3FF0ECDD0036A49ECAA
:1000C0000AF0F350016EF450026E400E011801E187
:1000D000025001E0ACD049EC0AF0F350016EF4504C
:1000E000026E490E011801E1025001E09ED049EC78
:1000F0000AF049EC0AF0D890035002E6200E035CA7
:1001000018E21F0E03140001E06FE16B800B01E0A9
:10011000E169050EE103F3CFE1F0E003F3CFE0F096
:10012000F450E127000EE025046E020EE121056E79
:1001300035D0D890035002E6400E035C18E21F0E43
:1001400003140001E06FE16B800B01E0E169050E33
:10015000E103F3CFE1F0E003F3CFE0F0F450E12767
:10016000000EE025046E010EE121056E17D01F0E72
:1001700003140001E06FE16B800B01E0E169050E03
:10018000E103F3CFE1F0E003F3CFE0F0F450E12737
:10019000000EE025046E000EE121056E49EC0AF028
:1001A000F350E66E04EBE9FF05EBEAFFE552E7509A
:1001B000EF6E49EC0AF0F350E66E04EBE9FF05EB55
:1001C000EAFFEE52E552E750EF6E49EC0AF049ECD7
:1001D0000AF0F350E66E04EBE9FF05EBEAFF020ECE
:1001E000E926000EEA22E552E750EF6E49EC0AF0EC
:1001F000F350E66E04EBE9FF05EBEAFF030EE92698
:10020000000EEA22E552E750EF6E49EC0AF0F35097
:10021000E66E04EBE9FF05EBEAFF040EE926000EAB
:10022000EA22E552E750EF6E0CD0FF0E14D00B0E11
:10023000011801E1025003E103500DD002D0FF0E7E
:100240000AD0032AD890035002E6500E035C02E362
:10025000FF0E01D034D746E9E7CFD9FF1200D9CF3E
:10026000E6FFE1CFD9FF83E9020E005C03E1000164
:10027000EA6918D0005016E101500001EA5D12E071
:10028000013410E2D890015002E60A0E015C0AE245
:1002900001EBE6FFE66A380EE66E92EC08F043E901
:1002A00001EBEAF041E9E7CFD9FF1200D9CFE6FF31
:1002B000E1CFD9FF85E941E8000408E000010250E0
:1002C000EC1902E10350ED1901E1EBD0000410E15B
:1002D000230EE66E500EE66EE66A92EC08F043E9F5
:1002E000240EE66E640EE66EE66A92EC08F043E9D0
:1002F000D880035004E79D0E025CFF0E035801E214
:10030000D0D0D890035004E6E80E025C030E0358E8
:1003100001E3C7D0033414E3015009E0210EE66E77
:10032000650EE66EE66A92EC08F043E908D0150E19
:10033000E66E650EE66EE66A92EC08F043E933D0AD
:10034000640ED89003BE03D0025C000E035827E36E
:10035000640EE66EE66A02EBE6FF03EBE6FF76EC80
:1003600019F0E552E5CFE1F0E7CFE0F00001E05110
:10037000056E01500AE0160E0524E66E650EE66E67
:10038000E66A92EC08F043E909D00A0E0524E66E0D
:10039000650EE66EE66A92EC08F043E904D0E66A80
:1003A000ADEC06F041E90A0ED89003BE03D0025C22
:1003B000000E035807E2033404E30250F608FF0E70
:1003C000035433E30A0EE66EE66AE66EE66A02EB73
:1003D000E6FF03EBE6FF76EC19F079EC19F0E55255
:1003E000E5CFE1F0E7CFE0F00001E051056E053424
:1003F00004E3FF0E0502F350056E01500BE0160EEC
:100400000524E66E650EE66E140EE66E92EC08F0BC
:1004100043E90AD00A0E0524E66E650EE66E140E58
:10042000E66E92EC08F043E905D0010EE66EADEC05
:1004300006F041E90250031018E00A0EE66EE66A83
:1004400002EBE6FF03EBE6FF79EC19F0E552E5CFAE
:10045000E1F0E7CFE0F00001E051056E053404E380
:10046000FF0E0502F350056E01D0056A01500BE046
:10047000160E0524E66E650EE66E280EE66E92EC0C
:1004800008F043E90AD00A0E0524E66E650EE66E12
:10049000280EE66E92EC08F043E902EBECF003EB79
:1004A000EDF042E9E7CFD9FF1200D9CFE6FFE1CF67
:1004B000D9FF84E941E8000408E000010150EC198B
:1004C00002E10250ED1901E186D100040CE1260E93
:1004D000E66E500EE66EE66A92EC08F043E9E66AD4
:1004E000ADEC06F041E9F10E011802E1D80E021858
:1004F00001E14AD10001ED3504E2EC510008000EA3
:10050000ED5502E2000411E1023404E2015000085A
:10051000000E02540AE2270EE66E640EE66E500EDE
:10052000E66E92EC08F043E919D0ED3504E2EC51A7
:100530000008000EED5502E3000410E1023404E26D
:1005400001500008000E025409E3280EE66E640E06
:10055000E66E500EE66E92EC08F043E9023404E2D7
:1005600001500008000E025464E2140EE66E650E9F
:10057000E66E1E0EE66E92EC08F043E90A0EE66E99
:10058000E66A640EE66EE66A01EBE6FF02EBE6FF62
:1005900076EC19F079EC19F0E552E5CFE1F0E7CF10
:1005A000E0F00001E051046E0A0E0424E66E650ED0
:1005B000E66E0A0EE66E92EC08F043E90A0EE66E6D
:1005C000E66AE66EE66A01EBE6FF02EBE6FF76EC32
:1005D00019F079EC19F0E552E5CFE1F0E7CFE0F062
:1005E0000001E051046E0A0E0424E66E650EE66E0C
:1005F000280EE66E92EC08F043E90A0EE66EE66A13
:1006000001EBE6FF02EBE6FF79EC19F0E552E5CFEE
:10061000E1F0E7CFE0F00001E051046E0A0E04249F
:10062000E66E650EE66E3C0EE66E92EC08F043E96F
:10063000AAD0023404E301509C08FF0E02542DE3BB
:10064000150EE66E650EE66EE66A92EC08F043E97A
:100650000A0EE66EE66A640EE66EE66AE668E6682C
:1006600001EBE6FF02EBE6FF4CEC1AF076EC19F03A
:1006700079EC19F0E552E5CFE1F0E7CFE0F00001C9
:10068000E051046E0A0E0424E66E650EE66E140E4A
:10069000E66E92EC08F043E91BD0023404E301500B
:1006A000F608FF0E02540DE3E66A57DB41E9150E2A
:1006B000E66E650EE66E140EE66E92EC08F043E907
:1006C00007D0E66A4ADB41E9010EE66E46DB41E906
:1006D000023404E30150F608FF0E025424E30A0E2C
:1006E000E66EE66AE66EE66AE668E66801EBE6FF55
:1006F00002EBE6FF4CEC1AF076EC19F079EC19F00D
:10070000E552E5CFE1F0E7CFE0F00001E051046E03
:100710000A0E0424E66E650EE66E280EE66E92EC76
:1007200008F043E911D0015002100AE0150EE66E00
:10073000650EE66E280EE66E92EC08F043E904D0F2
:10074000020EE66E0ADB41E90A0EE66EE66AE6682C
:10075000E66801EBE6FF02EBE6FF4CEC1AF079EC01
:1007600019F0E552E5CFE1F0E7CFE0F00001E0510C
:10077000046E0A0E0424E66E650EE66E3C0EE66E0E
:1007800092EC08F043E923D0150EE66E650EE66E96
:10079000E66A92EC08F043E9150EE66E650EE66E29
:1007A000140EE66E92EC08F043E9150EE66E650E47
:1007B000E66E280EE66E92EC08F043E9150EE66E42
:1007C000650EE66E3C0EE66E92EC08F043E901EB36
:1007D000ECF002EBEDF042E9E7CFD9FF1200D9CF00
:1007E000E6FFE1CFD9FF84E941E8000414E000010D
:1007F0000150EC1902E10250ED1901E1C2D00234BE
:1008000001E3BFD0D890025004E6100E015C270E21
:10081000025801E3B6D0000411E12A0EE66E500E34
:10082000E66EE66A92EC08F043E92B0EE66E640E83
:10083000E66E500EE66E92EC08F043E9D890025056
:1008400004E6E80E015C030E025821E30A0EE66E90
:10085000E66AE80EE66E030EE66E01EBE6FF02EBDB
:10086000E6FF76EC19F079EC19F0E552E5CFE1F00E
:10087000E7CFE0F00001E051046E0A0E0424E66EBA
:10088000650EE66EE66A92EC08F043E903D0E66A8C
:1008900064DA41E9640ED89002BE03D0015C000E18
:1008A000025821E30A0EE66EE66A640EE66EE66A18
:1008B00001EBE6FF02EBE6FF76EC19F079EC19F0BC
:1008C000E552E5CFE1F0E7CFE0F00001E051046E42
:1008D0000A0E0424E66E650EE66E140EE66E92ECC9
:1008E00008F043E904D0010EE66E37DA41E90A0E5A
:1008F000D89002BE03D0015C000E025820E30A0E1D
:10090000E66EE66AE66EE66A01EBE6FF02EBE6FFFC
:1009100076EC19F079EC19F0E552E5CFE1F0E7CF8C
:10092000E0F00001E051046E0A0E0424E66E650E4C
:10093000E66E280EE66E92EC08F043E904D0020E53
:10094000E66E0BDA41E90A0EE66EE66A01EBE6FFB7
:1009500002EBE6FF79EC19F0E552E5CFE1F0E7CFE5
:10096000E0F00001E051046E0A0E0424E66E650E0C
:10097000E66E3C0EE66ED6DB43E901EBECF002EBF3
:10098000EDF042E9E7CFD9FF1200D9CFE6FFE1CF82
:10099000D9FF84E941E8000407E000010150EC19A7
:1009A00002E10250ED195AE02C0EE66E640EE66E7E
:1009B000E66AB8DB43E90A0EE66EE66AE80EE66E22
:1009C000030EE66E01EBE6FF02EBE6FF76EC19F0B4
:1009D00079EC19F0E552E5CFE1F0E7CFE0F0000166
:1009E000E051046E160E0424E66E650EE66E2F0EC0
:1009F000E66E98DB43E90A0EE66EE66A640EE66E82
:100A0000E66A01EBE6FF02EBE6FF76EC19F079EC23
:100A100019F0E552E5CFE1F0E7CFE0F00001E05159
:100A2000046E160E0424E66E650EE66E430EE66E48
:100A300079DB43E9160EE66E650EE66E570EE66E3E
:100A400071DB43E9160EE66E650EE66E6B0EE66E22
:100A500069DB43E901EBECF002EBEDF042E9E7CFB3
:100A6000D9FF1200D9CFE6FFE1CFD9FF82E941E8F3
:100A7000003409E2003402E20050090804E3300EB9
:100A80000024026E12D0D890005002E60A0E005CDC
:100A90000AE3003402E200500F0805E3410E00248F
:100AA000F60F026E02D02D0E026E025000D042E907
:100AB000E7CFD9FF1200D9CFE6FFE1CFD9FF85E913
:100AC00044E8000407E000010250EC1902E1035081
:100AD000ED194FE0310EE66E3A0EE66EE66ADF0E75
:100AE000E66E370EE66E010EE66E0D0EE66EE66AF7
:100AF000D4DB48E9000103EBE0F0E16B070EE01501
:100B0000E66EB0DF41E9056E000102380F0BE06FC1
:100B10000338F00BE01303380F0BE16F0F0EE015F5
:100B2000E66EA0DF41E9066E0F0E0214E66E9ADF54
:100B300041E9076E086A013409E2013402E201501A
:100B4000020804E301EBE6FF31D941E9D950050F72
:100B5000E66EDACFE6FFE668E668010EE66E0D0E99
:100B6000E66E030EE66EE0DB47E902EBECF003EB2A
:100B7000EDF045E9E7CFD9FF1200D9CFE6FFE1CF8D
:100B8000D9FF85E952E8000417E12D0EE66E500EFC
:100B9000E66EE66AC7DA43E9200EE66E3A0EE66EC6
:100BA000E66ADF0EE66E370EE66E010EE66E0E0E9C
:100BB000E66EE66A72DB48E9056A0150055C53E2BD
:100BC00005EBE4F00001E56BE4BFE569E4510224C4
:100BD000E96EE5510320EA6EEF380F0B0F0BE66E5E
:100BE00041DF41E9E66E0001D950060FE06FDACF30
:100BF000E1F00550E824E26FE36B800B01E0E3696C
:100C0000E051E225E96EE151E321EA6EE552E75059
:100C1000EF6E05EBE4F0E56BE4BFE569E451022417
:100C2000E96EE5510320EA6EEF500F0BE66E1ADF16
:100C300041E9E66E0001D950060FE06FDACFE1F02E
:100C40000550E824010FE26FE36B800B01E0E369DC
:100C5000E051E225E96EE151E321EA6EE552E75009
:100C6000EF6E052AAAD7D890055002E6080E055C5B
:100C70002CE20001D950060FE06FDACFE1F0055009
:100C8000E824E26FE36B800B01E0E369E051E225C9
:100C9000E96EE151E321EA6E200EEF6ED950060FA6
:100CA000E06FDACFE1F00550E824010FE26FE36B6B
:100CB000800B01E0E369E051E225E96EE151E321B7
:100CC000EA6E200EEF6E052ACED7166A4F0EE66E3C
:100CD000EBDB41E9010EE66EE7DB41E9F2DBD950DF
:100CE000060FE66EDACFE6FFE668E668010EE66E0E
:100CF0000F0EE66EE66A18DB47E94F0EE66ED4DBB0
:100D000041E9E66AD1DB41E9DCDB53E9E7CFD9FF12
:100D10001200290EE66E640EE66E570EE66E02DADB
:100D200043E91200720EE66EBFDB41E9E66ABCDB06
:100D300041E9640EE66EB8DB41E97F0EE66EB4DB96
:100D400041E97F0EE66EB0DB41E9E66AADDB41E9E1
:100D5000E66AAADB41E961EF0AF0D9CFE6FFE1CF0D
:100D6000D9FF82E9140E0002F350006E720EE66E97
:100D70009BDB41E900EBE6FF97DB41E9640EE66EA1
:100D800093DB41E9140E0024E66E8EDB41E97F0E11
:100D9000E66E8ADB41E9E66A87DB41E9E66A84DBE5
:100DA00041E98FDB41E9E7CFD9FF1200D9CFE6FF58
:100DB000E1CFD9FF82E9080E0002F350170F006E51
:100DC000720EE66E71DB41E900EBE6FF6DDB41E997
:100DD000670EE66E69DB41E9080E0024E66E64DB0F
:100DE00041E96F0EE66E60DB41E9F80EE66E5CDB12
:100DF00041E9E66A59DB41E964DB41E9E7CFD9FF24
:100E00001200D9CFE6FFE1CFD9FF84E941E8000421
:100E100007E000010150EC1902E10250ED1972E007
:100E2000250EE66E640EE66EE66A7CD943E9640E32
:100E3000D89002BE03D0015C000E02581FE30A0ED8
:100E4000E66EE66A640EE66EE66A01EBE6FF02EB2A
:100E5000E6FF76EC19F079EC19F0E552E5CFE1F018
:100E6000E7CFE0F00001E051046E160E0424E66EB8
:100E7000650EE66E430EE66E55D943E90A0ED8902C
:100E800002BE03D0015C000E02581EE30A0EE66E9D
:100E9000E66AE66EE66A01EBE6FF02EBE6FF76EC59
:100EA00019F079EC19F0E552E5CFE1F0E7CFE0F089
:100EB0000001E051046E160E0424E66E650EE66E27
:100EC000570EE66E2FD943E90A0EE66EE66A01EB8D
:100ED000E6FF02EBE6FF79EC19F0E552E5CFE1F031
:100EE000E7CFE0F00001E051046E160E0424E66E38
:100EF000650EE66E6B0EE66E15D943E901EBECF07C
:100F000002EBEDF042E9E7CFD9FF12002E0EE66EBC
:100F1000480EE66EE66A06D943E91200D9CFE6FF2D
:100F2000E1CFD9FF83E944E8020E005C03E1000150
:100F3000EB69BCD0000408E0005001E0B7D00150DC
:100F40000001EB5D01E1B2D07F0E0114036E0334AA
:100F500002E20350340802E2340E036E2E0EE66EF7
:100F60003D0EE66E020EE66EDDD843E9700EE66ECB
:100F70009BDA41E9010EE66E97DA41E9A2DA720ED8
:100F8000E66E92DA41E9E66A8FDA41E9470EE66EEB
:100F90008BDA41E9350EE66E87DA41E94F0EE66EEF
:100FA00083DA41E9370EE66E7FDA41E9DF0EE66E5D
:100FB0007BDA41E986DA700EE66E76DA41E9E66AB6
:100FC00073DA41E97EDA720EE66E6EDA41E9010EFD
:100FD000E66E6ADA41E9480EE66E66DA41E903EB4D
:100FE000E6FF62DA41E94E0EE66E5EDA41E901AEF5
:100FF00008D0F80EE66E58DA41E9E66A55DA41E9BA
:1010000008D0030EE66E50DA41E9E00EE66E4CDAE7
:1010100041E957DAD890035002E6340E035C1BE234
:10102000720EE66E41DA41E90328E66E3DDA41E9E7
:10103000480EE66E39DA41E9340EE66E35DA41E9FA
:101040004E0EE66E31DA41E9E66A2EDA41E9E66AE9
:101050002BDA41E936DA7F0E01140001E06FE16B13
:10106000800B01E0E169E0C0E6FFE1C0E6FF1C0E95
:10107000E66E3A0EE66EE66AD950040FE66EDACFF7
:10108000E6FF50EC1CF047E9D950040FE66EDACFCA
:10109000E6FFDF0EE66E370EE66EE66A090EE66ED6
:1010A000040EE66E41D947E901EBEBF045E9E7CFE5
:1010B000D9FF1200D9CFE6FFE1CFD9FF82E9003492
:1010C00002E200500F0802E20F0E006E590EE66EAB
:1010D000EBD941E9020EE66EE7D941E900EBE6FF04
:1010E000E3D941E9EED941E9E7CFD9FF1200590E22
:1010F000E66EDAD941E9030EE66ED6D941E9E66A31
:10110000D3D941E961EF0AF0590EE66ECDD941E934
:10111000030EE66EC9D941E9010EE66EC5D941E973
:1011200061EF0AF0D9CFE6FFE1CFD9FF84E942E8C9
:10113000D890005002E6200E005C18E21F0E00144A
:101140000001E06FE16B800B01E0E169050EE10356
:10115000F3CFE1F0E003F3CFE0F0F450E127000E2D
:10116000E025046E020EE121056E35D0D8900050C6
:1011700002E6400E005C18E21F0E00140001E06F52
:10118000E16B800B01E0E169050EE103F3CFE1F0D3
:10119000E003F3CFE0F0F450E127000EE025046E09
:1011A000010EE121056E17D01F0E00140001E06F43
:1011B000E16B800B01E0E169050EE103F3CFE1F0A3
:1011C000E003F3CFE0F0F450E127000EE025046ED9
:1011D000000EE121056E400EE66E66D941E9490E2A
:1011E000E66E62D941E902EBE6FF5ED941E901EB27
:1011F000E6FF5AD941E904EBE9FF05EBEAFFEFCF3F
:10120000E6FF52D941E904EBE9FF05EBEAFFEE52B4
:10121000EFCFE6FF49D941E9100EE66E45D941E925
:1012200004EBE9FF05EBEAFF020EE926000EEA22D5
:10123000EFCFE6FF39D941E904EBE9FF05EBEAFF1F
:10124000030EE926000EEA22EFCFE6FF2DD941E991
:1012500004EBE9FF05EBEAFF040EE926000EEA22A3
:10126000EFCFE6FF21D941E92CD9000904E00001C4
:10127000010EE96F02D00001E96B43E9E7CFD9FF26
:101280001200450EE66E10D941E91BD90001EA6B48
:101290000F0EEC6F270EED6F1200D9CFE6FFE1CFF6
:1012A000D9FF89E9730EE66EFFD841E907EBE6FF47
:1012B000FBD841E906EBE6FFF7D841E905EBE6FF8D
:1012C000F3D841E9000104EBE0F0E16BE0C0E6FF98
:1012D000EBD841E9FF0E0314E66EE6D841E900EBD6
:1012E000F6FF01EBF7FF02EBF8FF0800F55014E002
:1012F000D9CFE9FFDACFEAFFEFCFF6FFEE2AEFCF43
:10130000F7FF000EEE22EFCFF8FFEE220800F5CF38
:10131000E6FFCAD841E9E3D7E66AC6D841E9D1D8A1
:1013200041E9E7CFD9FF1200D9CFE6FFE1CFD9FFDE
:1013300088E9730EE66EB8D841E906EBE6FFB4D84B
:1013400041E905EBE6FFB0D841E904EBE6FFACD894
:1013500041E9000103EBE0F0E16BE0C0E6FFA4D857
:1013600041E9FF0E0214E66E9FD841E900EBE9FF68
:1013700001EBEAFFEF500CE000EBE9FF01EBEAFFC5
:10138000002A000E0122EFCFE6FF8ED841E9EED70A
:10139000E66A8AD841E995D841E9E7CFD9FF12003A
:1013A000400EE66E81D841E9690EE66E7DD841E9CE
:1013B00088D8000903E0FF0E03D002D0000E00D051
:1013C0001200D9CFE6FFE1CFD9FF85E9400EE66EE6
:1013D0006BD841E9410EE66E67D841E900EBE0F0D9
:1013E00001EBE1F002EBE2F003EBE3F0180E000199
:1013F000D890E333E233E133E033E806F9E100016A
:10140000E051E66E51D841E900EBE0F001EBE1F08C
:1014100002EBE2F003EBE3F0100E0001D890E333AF
:10142000E233E133E033E806F9E10001E051E66E32
:101430003BD841E900EBE0F001EBE1F002EBE2F038
:1014400003EBE3F0080E0001D890E333E233E1331D
:10145000E033E806F9E10001E051E66E25D841E904
:1014600000EBE0F001EBE1F002EBE2F003EBE3F084
:101470000001E051E66E18D841E923D8000903E0E5
:10148000FF0E03D002D0000E00D041E9E7CFD9FF14
:101490001200400EE66E08D841E9720EE66E04D8DE
:1014A00041E92FD800D01200D9CFE6FFE1CFD9FF14
:1014B00082E9ACA2FED700EBADFF41E9E7CFD9FF4F
:1014C0001200D9CFE6FFE1CFD9FF81E942E819D870
:1014D000F350016EF450026E023405E30001010E78
:1014E000E86FFF0E0AD0060E011801E1025003E179
:1014F000000E03D002D0FF0E00D043E9E7CFD9FFA2
:101500001200D9CFE6FFE1CFD9FF81E941E8000120
:101510000B0ED96F9EBA06D0D95103E1F368F46877
:101520000FD0F8D79E9AAE50016E01EBE0F00001AB
:10153000E16BE0BFE169E0C0F3FFE1C0F4FF00D080
:0815400042E9E7CFD9FF1200D8
:08154800D9CFE6FFE1CFD9FF86
:1015500081E94BE8E8EC1BF09EEC11F0F6EC10F0A2
:10156000F3CFA6F0F4CFA7F00001D890A75104E67E
:10157000340EA65D210EA75909E20001D890A751AB
:1015800004E6DC0EA65D050EA7590CE2700EE66EB1
:10159000170EE66E1BEC11F042E90001700EA66F0B
:1015A000170EA76F34EC11F00001AA6FAB6B800B24
:1015B00001E0AB690001AB3504E2AA519608000EC8
:1015C000AB5509E3320E0001D890ABBF03D0AA5D42
:1015D000000EAB5909E2600EE66E3AEC11F041E9FB
:1015E000600E0001AA6FAB6B49EC11F00001E06FD7
:1015F000040E0001E05D04E3E66A4FEC11F041E9FE
:101600005EEC11F0F3CFB3F0F4CFB4F00001B351BE
:10161000FF08070EB45509E2000EE66EE66A84EC98
:1016200011F042E90001B36BB46B0EEC00F041EC39
:1016300009F0D0EC09F00001E06F0001E03517E39C
:10164000090EE66E3A0EE66EE66AE668E668E66A57
:101650000C0EE66E020EE66E4DEC09F048E9000154
:10166000140ED96F0001D95101E0FCD7E2D74BEC41
:1016700000F00001E06F0001E03512E341EC09F0F9
:10168000F80EE66E390EE66EE66AE668E668E66A29
:101690000C0EE66E020EE66E4DEC09F048E9FFD73F
:1016A000B3EC15F00D01D48BE66AB3C0E6FFB4C00D
:1016B000E6FFE66AE66A140EE66E0F0EE66EE2ECF0
:1016C00017F047E9600EE66ED0EC17F041E9000133
:1016D000A06B0001280EDB6FCB0EE66E000EE66EEF
:1016E000CA0EE66E000EE66EC20EE66E000EE66EE6
:1016F000BE0EE66E000EE66ECEEC16F048E900096E
:1017000002E198EF0FF00001280EDB6F0001A051FD
:1017100004E0040E0001A05D3CE1C30E0001BE190F
:1017200006E1020EBF1903E1C05101E1C1512FE1F1
:101730000001CA052CE10001C2A320D03C0E00012B
:10174000D76FD86B2F0EE66EE66AE66A92EC08F069
:1017500043E9F20EE66E390EE66EE66AE66A800E40
:10176000E66E010EE66E0F0EE66E0B0EE66E4DECAB
:1017700009F048E90001020EA06F09D00001D7511D
:10178000D81105E177EC08F00001010EA06FA4D795
:10179000CFD3020E0001A05D31E10001D751D81175
:1017A0002BE1220EE66EE66AE66A92EC08F043E967
:1017B0000001030EA06F0001AC6B0001AF6B0001D4
:1017C000010EAE6F49EC11F00001A16F0001F10EA6
:1017D000A86FD80EA96F0001B26B0001BD6B0A6A39
:1017E000020EE66EE6682FEC01F042E9020EE66EAC
:1017F000E6688EEC07F042E96FD79AD30001A005A6
:1018000016E1C30E0001BE1906E1020EBF1903E185
:10181000C05101E1C15109E10001CA0506E1000121
:10182000C2A303D084EC08F089D756D781D3030E26
:101830000001A05D01E07CD3C30E0001BE1906E1EA
:10184000020EBF1903E1C05101E1C1510FE10001D6
:10185000CA050CE10001C2B308D041EC09F077ECF5
:1018600008F00001010EA06F37D71DD1800E0001D6
:10187000BE1906E1020EBF1903E1C05101E1C151D9
:101880002EE1080E0001CA5D2AE1040EE66EE66A4A
:10189000C5C0E2F0E2C0E3F00001E26B0001C45118
:1018A0000001E2110001E06FE3C0E1F0E0C0E6FFFB
:1018B000E1C0E6FFBEEC19F0E552E550026EE750DC
:1018C000016E0001A7350250A71904E6A651015C7C
:1018D000A751025802E3949401D09484E4D0400EBE
:1018E0000001BE1906E1050EBF1903E1C05101E177
:1018F000C1516CE1080E0001CA5D68E10A5059E06F
:10190000400E0001C21555E00F0E0001C215000186
:10191000A46F0001C9390F0B0001A56F020E000171
:10192000A35D05E10001A55102E1076A3BD0030E6A
:101930000001A35D07E10C0E0001A55D03E1010EAE
:10194000076E30D0040E0001A35D06E10001A55131
:1019500003E1020E076E26D0050E0001A35D09E02B
:10196000060E0001A35D05E00001A5510001A35D85
:1019700019E1010E0001E76EA51902E7A53502D0B5
:10198000A551E75C0FE2090E0001E76EA51902E719
:10199000E73402D0E750A55D05E2030E0001A5255E
:1019A000FE0F076EE66A07EBE6FF2FEC01F042E957
:1019B0000CD00F0E0001C2150001A26F0001C93941
:1019C0000F0B0001A36F010E0A6E6DD0880E00018F
:1019D000BE1906E1020EBF1903E1C05101E1C15178
:1019E00037E1080E0001CA5D33E10001A15130E189
:1019F000E80EE66E030EE66EE66AE66AF10EE66E45
:101A0000020EE66EE66AE66AC3C0E6FFE66AE66ACA
:101A1000E66A80EC1AF0FAEC19F0E552E5CFE3F053
:101A2000E5CFE2F0E5CFE1F0E7CFE0F0310E0001E5
:101A3000E05F000E0001E15B000E0001E25B000EC2
:101A40000001E35B0001E051036EE151046E2BD015
:101A5000350E0001BE1906E1060EBF1903E1C051A3
:101A600001E1C15108E1030E0001CA5D04E100017A
:101A7000C351086E18D0200E0001BE1906E1030EF6
:101A8000BF1903E1C05101E1C1510DE1080E000190
:101A9000CA5D09E10001C451096EE66A09EBE6FF7F
:101AA0008EEC07F042E9B3C0E0F0B4C0E1F0000111
:101AB000E26BE36BBE0EE96E000EEA6EEE500001C3
:101AC000E01908E1EE50E11905E1EE50E21902E1FA
:101AD000EE50E31924E1030E0001A15D20E10B6A41
:101AE0000001CA510B5C19E20BEBE9FFEA6AE9BE9F
:101AF000EA68C20EE926000EEA22EF50E66E0BEB12
:101B0000E9FFEA6AE9BEEA68B50EE926000EEA22B4
:101B1000E552E750EF6E0B2AE3D7CAC0BDF00001D3
:101B2000A1514EE10001AC511AE00001AE510EE0AE
:101B3000010EE66EAAC0E6FFABC0E6FF01EC07F0BF
:101B400043E90001280EAD6F0001AE6B0001AD51FD
:101B500005E10001AC6B0001010EAE6F30D0000159
:101B6000AB350450AB1904E6AA51035CAB510458E1
:101B700003E3010E0B6E01D00B6A0001AE5115E0BC
:101B8000010EE66E0BEBE6FF03EBE6FF04EBE6FF70
:101B900056EC01F044E9010EE66E09EBE6FF8EEC2F
:101BA00007F042E90001AE6B0AD0E66A0BEBE6FFF4
:101BB00003EBE6FF04EBE6FF56EC01F044E9B8D195
:101BC0000001A10501E0DED00001B13504E2B05111
:101BD0008108010EB1553EE2100EE66E270EE66E4C
:101BE000E66AE66A4E0EE66E0E0EE66EE66AE66A95
:101BF000B0C0E4F0B1C0E5F00001E66BE76BE5AF23
:101C000002D0E669E769810E0001E45F010E000180
:101C1000E55B000E0001E65B000E0001E75BE4C03F
:101C2000E6FFE5C0E6FFE6C0E6FFE7C0E6FF80ECC2
:101C30001AF0FAEC19F0E552E5CFE3F0E5CFE2F067
:101C4000E5CFE1F0E7CFE0F00001E051056EE151B2
:101C5000066E3DD0E80EE66E030EE66EE66AE66AB4
:101C6000850EE66E0A0EE66EE66AE66AB0C0E4F03D
:101C7000B1C0E5F00001E66BE76BE5AF02D0E669C5
:101C8000E769810E0001E45F010E0001E55B000ED3
:101C90000001E65B000E0001E75BE4C0E6FFE5C083
:101CA000E6FFE6C0E6FFE7C0E6FF80EC1AF0FAECDC
:101CB00019F0E552E5CFE3F0E5CFE2F0E5CFE1F052
:101CC000E7CFE0F00001E051056EE151066E000142
:101CD0000634A951061804E60550A85D0650A95916
:101CE00004E205EBA8F006EBA9F00001AC512BE0F3
:101CF0000001AE511FE00001AF510AE0010EE66E97
:101D0000F10EE66ED80EE66E55EC02F043E909D00E
:101D1000010EE66EA8C0E6FFA9C0E6FF55EC02F092
:101D200043E989EC06F00001280EAD6F0001AE6BAF
:101D30000001AF6B0001AD5105E10001AC6B00018A
:101D4000010EAE6F1ED00001AE5113E0010EE66E23
:101D500005EBE6FF06EBE6FF55EC02F043E9010E6A
:101D6000E66E09EBE6FF8EEC07F042E90001AE6B90
:101D700008D0E66A05EBE6FF06EBE6FF55EC02F05D
:101D800043E9D6D0020E0001A15D48E10001AC514B
:101D90001AE00001AE510EE0010EE66EA6C0E6FFAD
:101DA000A7C0E6FFC5EC04F043E90001280EAD6FC3
:101DB0000001AE6B0001AD5105E10001AC6B00010B
:101DC000010EAE6F2AD00001AE5117E0010EE66E93
:101DD00001EBE6FF02EBE6FFEFEC03F043E9010E57
:101DE000E66E09EBE6FF8EEC07F042E9020E000119
:101DF000D76FD86B0001AE6B10D00001D751D8114E
:101E00000CE1E66A01EBE6FF02EBE6FFEFEC03F024
:101E100043E9020E0001D76FD86B8AD0030E000190
:101E2000A15D01E085D00001AC5148E00001AE5158
:101E300012E092EC06F0010EE66EB2C0E6FFB3C00F
:101E4000E6FFB4C0E6FF5BEC05F044E90001280EB4
:101E5000AD6F0001AE6B0001AD512FE10001B22B5F
:101E6000020E0001E76EB21902E7B23502D0B2519C
:101E7000E75C02E20001B26B800EE66ED0EC17F078
:101E800041E90D01D48BE66AB3C0E6FFB4C0E6FFBA
:101E9000E66AE66A140EE66E0F0EE66EE2EC17F0E6
:101EA00047E9600EE66ED0EC17F041E90001BD6B2A
:101EB0000001AC6B0001010EAE6F3AD00001AE51D3
:101EC00025E092EC06F0010EE66EE668B3C0E6FF90
:101ED000B4C0E6FF5BEC05F044E9010EE66EBDC060
:101EE000E6FFB50EE66E000EE66EBDEC05F044E9C9
:101EF000010EE66E09EBE6FF8EEC07F042E9010EFB
:101F00000001D76FD86B0001AE6B12D00001D75122
:101F1000D8110EE1E66ABDC0E6FFB50EE66E000E12
:101F2000E66EBDEC05F044E9010E0001D76FD86BF9
:101F30000001E95102E0AAEF0AF00001DB511DE1C6
:101F4000040E0001A05D19E041EC09F0DE0EE66E22
:101F5000390EE66EE66AE668E668E66A0C0EE66E3C
:101F6000020EE66E4DEC09F048E93C0E0001D76F19
:101F7000D86B0001040EA06F1AD00001DB5117E1ED
:101F8000040E0001A05D13E10001D751D8110FE14B
:101F900077EC08F0200EE66ED0EC17F041E9729E67
:101FA000F29AA38C0300A39C728EAAEF0AF06CEF46
:101FB0000BF04CE9E7CFD9FF1200640E0001A62711
:101FC000000EA723D890A75104E6980EA65D210E17
:101FD000A75904E3DC0EA66F050EA76FA6C0E6FFA7
:101FE000A7C0E6FF28D942E90001010EAC6FAE6F31
:101FF0001200020E0001AA25AA6F000EAB21AB6FE2
:10200000980ED890ABBF03D0AA5D000EAB5903E386
:10201000320EAA6FAB6BAAC0E6FF2CD941E90001D2
:10202000010EAC6FAE6F1200D9CFE6FFE1CFD9FF42
:1020300081E946E80001B451016E026A0F0E0116F3
:10204000000E0216B3390F0B036EB439F00B0312F6
:10205000B4390F0B046E0F0E0316000E04160F0E8C
:10206000B315056E066A0001D950010FE06FDACF93
:10207000E1F0B2C0E2F0E36BE2BFE369D890E2378F
:10208000E337E051E225E96EE151E321EA6EEE2A01
:10209000000EEF2201EBE3F0E26BE2170F0EE31705
:1020A0000438F00BE56F03380F0BE5130338F00B22
:1020B000E46FF00EE417000EE517E251E425E06F3F
:1020C000E351E521E16F0F0E0514E66FE76BE05178
:1020D000E6250001B36F0001E151E7210001B46F73
:1020E000B3C0E6FFB4C0E6FF0FD942E947E9E7CF46
:1020F000D9FF1200030E0001A05D0DE1A12B040E1B
:10210000A15D01E1A16BA1C0E6FFC9D841E90001D1
:10211000AC6B010EAE6F1200030E0001A05D1EE15C
:10212000A10505E1AC0503E1010EAF6F13D0A1518C
:1021300004E1AC0502E15DDF0DD0020EA15D04E11A
:10214000AC0502E13ADF06D0030EA15D03E1AC0568
:1021500001E16ADF0001010EAC6FAE6F1200D9CF52
:10216000E6FFE1CFD9FF83E941E8A69CA69EA684BD
:10217000AA6A01EBA9FF00EBA8FFF250800B01E077
:10218000010E036EF29E550EA76EAA0EA76EA682D2
:10219000A6A202D0FDD7FCD7A198A6940350E8B020
:1021A000F28EE8A0F29E42E9E7CFD9FF1200D9CF24
:1021B000E6FFE1CFD9FF82E942E8A69CA69EAA6A83
:1021C00000EBA9FFF250800B01E0010E026EF29EBF
:1021D000A680A850036E0250E8B0F28EE8A0F29EEE
:1021E000035000D043E9E7CFD9FF1200010EE66E9D
:1021F000DEDF41E90001E26FE36B800B01E0E369A0
:10220000E2C0E3F0E26BE2C0E6FFE3C0E6FFE66AAD
:10221000CEDF41E9E552E7CFE3F0E552E7CFE2F068
:102220000001E211E06FE3C0E1F0E0C0F3FFE1C0C4
:10223000F4FF00D01200D9CFE6FFE1CFD9FF83E948
:10224000FF0E0014E66EE66A8ADF42E9000101EB48
:10225000E0F0E16BE0C0E6FF010EE66E80DF42E9F0
:1022600041E9E7CFD9FF1200020EE66EA0DF41E997
:1022700000D01200D9CFE6FFE1CFD9FF82E900EB11
:10228000E6FF020EE66E6BDF42E941E9E7CFD9FFD8
:102290001200030EE66E8BDF41E900D01200D9CFA9
:1022A000E6FFE1CFD9FF82E900EBE6FF030EE66E21
:1022B00056DF42E941E9E7CFD9FF1200050EE66E8D
:1022C00076DF41E90001E26FE36B800B01E0E36937
:1022D000E2C0E3F0E26BE2C0E6FFE3C0E6FF040E1B
:1022E000E66E65DF41E9E552E7CFE3F0E552E7CF7F
:1022F000E2F00001E211E06FE3C0E1F0E0C0F3FFC3
:10230000E1C0F4FF00D01200D9CFE6FFE1CFD9FF42
:1023100083E9FF0E0014E66E040EE66E20DF42E94C
:10232000000101EBE0F0E16BE0C0E6FF050EE66EB8
:1023300016DF42E941E9E7CFD9FF120094849E0EEF
:10234000CB6E070ECA6E0C0EBD6E4F0EBE6E120027
:1023500090DB86E90150010600090CE002EBE6FF84
:1023600003EBE6FF00EBE6FF69DBF4E1E11DF2E1E0
:10237000010E01D0000E41E9E5CFDAFFE7CFD9FF2A
:10238000120077DB89E97BE80A6A0B6A02EBF6FF49
:1023900003EBF7FF04EBF8FF0800F550096E095056
:1023A00001E12DD3250E095C01E01BD30C6A0D6AF7
:1023B0000E6A0F6A106A2DDB2D0E095C0CE02B0EE5
:1023C000095C09E0200E095C06E0230E095C03E0CD
:1023D000300E095C15E10950300A10E0130A0CE0D8
:1023E000030A08E00B0A04E0060AE5E10C80E3D7E3
:1023F0000C82E1D70C84DFD70C86DDD70C88DBD7C5
:102400002A0E095C13E1A5DB0DE30C801CEBE0F068
:102410001DEBE1F00001E06DE11F000EE123E05152
:102420000D6E02D09CEB0DF0F4DA07D0126A3FDBA0
:1024300002E06BDBFCD792EB0DF00CB00C982E0E8B
:10244000095C15E1E6DA2A0E095C08E182DB04E2A8
:102450009CEB0EF0010E0F6EDCDA09D0126A27DB5E
:1024600002E053DBFCD792EB0EF0010E0F6E680E0C
:10247000095C07E1CEDA680E095C1DE1030E106EFF
:1024800019D0740E095C16E07A0E095C13E0480E50
:10249000095C06E0540E095C03E05A0E095C02E197
:1024A000020E07D06C0E095C03E06A0E095C03E1C2
:1024B000010E106EAEDA09506E0A01E16ED21E0AEC
:1024C00001E128D1200A01E125D13F0A01E1FDD037
:1024D0001A0A01E1FAD00D0A01E1F7D0200A01E160
:1024E000F4D03A0A01E1F1D0200A01E1EED0260A47
:1024F00001E1EAD00D0A01E1E7D01A0A01E19ED01C
:10250000200A3BE0300A1AE0460A0EE0250A01E004
:1025100072D2D950020FE96E000EDA20EA6E010E77
:10252000EE5E000EEE5AEE5A0FDB250EE66E86DAF0
:1025300003E1E11D01E159D20A2A5BD2116A0D5073
:10254000010803E20D04116EF5DA115007E0010EE7
:102550000C1404E16DDA01E048D2116AD3DAEF50CD
:10256000096ECBDA03E1E11D01E13FD20A2A000E38
:102570000B225EDA01E13FD238D2020E105C08E194
:10258000030E4EDAEE50176EEE50186EEF5007D075
:10259000E7DAE26BE051176EE151186EE251196E05
:1025A00017EBE6FF18EBE6FF19EBE6FF97EC1CF0E4
:1025B00043E9EEC0E0F0EFC0E1F0F0C0E2F000016E
:1025C000E0511C6EE1511D6E0F5006E01C500E5C78
:1025D00003E20E501C6E1D6A1C500D5C02E29CEB67
:1025E0000DF050DA05E00D500E5C02E28EEB0DF0BE
:1025F0000CB004D01DDA01E0F8D1116A126A17EBB1
:10260000F6FF18EBF7FF19EBF8FF0800F550096E1D
:10261000095010E00D50125C0DE26FDA03E1E11D8C
:1026200001E1E3D10A2A000E0B22122AD950170F1A
:1026300055DAEBD7FDD901E1DED1D7D163DAEE501F
:102640001A6EED501B6E1AEBE6FF1BEBE6FF89ECF2
:102650001CF042E9F3501C6EF4501D6E0F5006E062
:102660001C500E5C03E20E501C6E1D6A1C500D5C6B
:1026700002E29CEB0DF006DA05E00D500E5C02E282
:102680008EEB0DF00CB004D0D3D901E0AED1116ABD
:10269000126A1AEBE9FF1BEBEAFFEF50096E0950D3
:1026A0000FE00D50125C0CE228DA03E1E11D01E1BC
:1026B0009CD10A2A000E0B22122A1A2A1B22E9D7C1
:1026C000B7D901E198D191D10C8E10040AE1040E22
:1026D000A7D9EE50136EEE50146EEE50156EEF50FB
:1026E00032D0030E105C16E10CAE0CD00BDAEFCF3B
:1026F000E0F00001E16BE26BE36BE0AF23D0E16956
:10270000E2691FD0FFD9EFCFE0F00001E051136E76
:10271000146A20D0020E105C0CE10CAE06D0030E41
:102720007FD9B6D9E2AF0ED00CD0030E79D9B0D98B
:1027300009D00CAE0AD014DAE26BE36BE1AF02D041
:10274000E269E369BCD9166E07D00ADAE051136E6C
:10275000E151146E156A166A0F5002E1010E0E6EF9
:102760001E6A1F6AD950400FE66E000EDA20E66E30
:10277000E552E550436EE750426E416A116A0A0E17
:10278000106E0950780A12E0200A10E0280A0CE0C6
:10279000200A0AE03F0A06E00D0A02E0200A08E1EA
:1027A000020E05D0080E03D0080E0926100E106E7A
:1027B0000CBE02D00C920C94800E0C1417E0163450
:1027C00015E3E668E668E668E66842D980EC1AF048
:1027D000E552E5CFE3F0E5CFE2F0E5CFE1F0E7CF7A
:1027E000E0F000016CD9166E2D0E07D00CA202D0BD
:1027F0002B0E03D00CA404D0200E206E1E2A01D074
:10280000206A0E5005E1135014101510161061E0E7
:102810000001B00EE06F3A0EE16F000EE26F83D957
:10282000E0EC1AF0E552E5CFE6F0E5CFE5F0E5CFD4
:10283000E4F0E7CFE3F00001E051E325F36EE1516E
:10284000E421F46EE251E521F86EF4CFF7FFF3CF07
:10285000F6FF0800F550126E580E095C05E1610E96
:10286000125C02E3200E125E5ED9DDEC1AF0E55236
:10287000E550166EE550156EE550146EE750136E78
:1028800042EBE9FF43EBEAFF4206000E435A12EB2C
:10289000EFFF1E2A1350141015101610B9E10CA6E4
:1028A00019D06F0E095C06E10E501E5C13E31E2862
:1028B0000E6E10D0780E095C09E0580E095C06E037
:1028C000620E095C03E0420E095C04E1020E1F6E19
:1028D00001D01E6A100E0C1407E00D500E5C04E2CD
:1028E0000F5002E18DEB0EF00E501E5C03E21E5005
:1028F0000E5E01D00E6A0E501E241F24D8800D5487
:1029000007E20E500D5CD8801E54D8801F54116E03
:10291000010E0C1406E1115004E08AD866E10AD9D0
:10292000116A205007E010D920EBE6FF87D802E1BA
:10293000E11D5BE01F500BE007D9300EE66E7ED83C
:1029400002E1E11D52E0D9D802E1E11D4EE00E5056
:102950001F5C02E21F500E5E300EE66E0EEBE6FFCD
:10296000DCD843E1422A000E432242EBE9FF43EB6D
:10297000EAFFEF50126E125008E0E6D812EBE6FFC5
:102980005DD8F0E1E11DEEE130D052D82EE10E50DD
:102990001E2411241F240A262CD01050030A1CE0E8
:1029A000010A14E0030A07E0ADD8C9D80AEBEEFF2C
:1029B0000BEBEDFF20D08BD8E36BE1AF02D0E269E7
:1029C000E369A0D84ED8E3C0EEFF15D080D8E1BFB0
:1029D000E26998D846D80FD095D8B1D80AEBEFFF66
:1029E0000AD08BD805E1E11D03E1F368F4680BD050
:1029F0000A2A000E0B22D950020F70D8CDD40AEB50
:102A0000F3FF0BEBF4FF7CE9E5CFDAFFE7CFD9FF6B
:102A10001200D950020F62D80800F550096E12005A
:102A2000005E000E015A00EBE9FF01EBEAFF120025
:102A3000200EE66E11EBE6FF8DEF15F0BCEC1CF0FE
:102A400043E9F3CFE0F0F4CFE1F00001F31C120012
:102A500013EBE6FF14EBE6FF15EBE6FF16EBE6FFE4
:102A600012006DD8E0C0EEFFE1C0EEFFE2C0EEFF65
:102A70001200D9CFE6FFDACFE6FFE1CFD9FFE2CFF0
:102A8000DAFF12001C500D5C116E54D80F5012006A
:102A9000EECFE0F0EECFE1F0EFCFE2F00001E36B3C
:102AA0001200EECFE0F0EFCFE1F00001120009508C
:102AB000E66EE66A1BEC1DF042E9F3501200E051AD
:102AC000136EE151146EE251156EE35112000AEBE0
:102AD000E0F00BEBE1F00001E26B1200E96E000E9A
:102AE000DA20EA6EEF2AEECFF6FF000EEF22EECFED
:102AF000F7FFEF22EECFF8FF120026D809EBE6FF32
:102B00001EEF15F0020E10EF15F00A0E1202F35030
:102B10000924D00F126E09EF15F016D8A8EC11F0A9
:102B200044E90009120010EBE6FFE66AE66AE66A8D
:102B300028EF15F011500A26000E0B221200EE505D
:102B4000EFCFEAFFE96E120005EBE6FF06EBE6FFCA
:102B50001200D8DFEE501C6EED501D6E1D341200B9
:062B6000D1DF51EF15F07A
:0A2B6600800EE66E1ADA41E9030E54
:102B7000706EA00E716E820E726E100E736E779E66
:102B8000778C606A0F01506B0E01206B306B406BCD
:102B9000506B606B706B0D01F86B0F01500E006F86
:102BA000016B510E046F056BA80E086F096BC60E02
:102BB0000C6FA00E0D6F580E106F600E116F146B1E
:102BC000156B0D01640E606F616B646B656BD4698E
:102BD000D56B320EE06F450EE16F670EE26FE36B6F
:102BE000E46BE56BE66BE76BF06BF16BF26BF26B32
:102BF0000F011869E00E196F19971C6B1D6B1D975B
:102C00001200D9CFE6FFE1CFD9FF89E95AE8400E9B
:102C10000F6E0F0E106E300E116E0F0E126E200E14
:102C2000136E0F0E146E200E156E0E0E166E300EF5
:102C3000176E0E0E186E400E196E0E0E1A6E500E96
:102C40001B6E0E0E1C6E600E1D6E0E0E1E6E700E36
:102C50001F6E0E0E206E0D01F8417F0B226E096A69
:102C6000080E095C01E394D00001D9500F0FE06F0A
:102C7000DACFE1F00950020DE051F324E96EE151A1
:102C8000F420EA6EEE500B6EED500C6E8BEB0DF0F7
:102C90008CEB0EF0095002080BE222902242D95030
:102CA000220FE96EDACFEAFFEF50010B01E16ED09F
:102CB0000BEBE9FF0CEBEAFFEF50080B67E1FC0EB2
:102CC000E06F0BEBE9FF0CEBEAFFE051EF16030EB0
:102CD0000014E06F0BEBE9FF0CEBEAFFE051EF12A1
:102CE00000AC04D0400E0110216E02D081EB21F027
:102CF000050E0B24E96E000E0C20EA6E21EBEFFFAF
:102D000000AA03D0010E216E01D0216A21EBE6FF5B
:102D100004EBE6FF05EBE6FF06EBE6FF07EBE6FF5D
:102D20000B28E06F000E0C20E16FE0C0E6FFE1C071
:102D3000E6FF48D947E9060E0B26000E0C220A6A68
:102D400001500A5C15E202EBE9FF03EBEAFF022AFD
:102D5000000E0322EF50E66E0BEBE9FF0CEBEAFFEF
:102D60000B2A000E0C22E552E750EF6E0A2AE8D734
:102D70000DEBE9FF0EEBEAFFEF50040B05E10DEB65
:102D8000E9FF0EEBEAFFEF86010E04D0092A68D7AF
:102D9000000E00D05BE9E7CFD9FF1200D9CFE6FFE4
:102DA000E1CFD9FF89E946E80001F26B60AE05D0BA
:102DB000600E096E0F0E0A6E58D00F0150AF05D08D
:102DC000500E096E0F0E0A6E50D00D01F851040B13
:102DD00009E10E012051800B05E0200E096E0E0E58
:102DE0000A6E43D00D01F851080B09E10E01305174
:102DF000800B05E0300E096E0E0E0A6E36D00D0106
:102E0000F851100B09E10E014051800B05E0400E16
:102E1000096E0E0E0A6E29D00D01F851200B09E142
:102E20000E015051800B05E0500E096E0E0E0A6E19
:102E30001CD00D01F851400B09E10E016051800BCF
:102E400005E0600E096E0E0E0A6E0FD00D01F851EE
:102E5000800B09E10E017051800B05E0700E096EC8
:102E60000E0E0A6E02D0000E97D009EBE9FF0AEBB6
:102E7000EAFFEF501F0B0001F26FA49274AC07D071
:102E800000D000EBE9FF01EBEAFFEF86749C89EBD1
:102E90000BF08AEB0CF000EBE9FF01EBEAFFEF6AC5
:102EA000050E0924E96E000E0A20EA6EEF500E6E40
:102EB0000F0E0E14E66E02EBE9FF03EBEAFFE5529C
:102EC000E750EF6ED9500E0FE96EDACFEAFFEF5000
:102ED000400B05E000EBE9FF01EBEAFFEF8C020E8F
:102EE0000924E96E000E0A20EA6EEF500E6ED950EA
:102EF0000E0FE96EDACFEAFFEF50080B08E000EBA7
:102F0000E9FF01EBEAFFEF8A010E0E6E01D00E6AB7
:102F10000EEBE6FF06EBE6FF07EBE6FF00010928F4
:102F2000E06F000E0A20E16FE0C0E6FFE1C0E6FFBF
:102F300008D945E9060E0926000E0A2202EBE9FF30
:102F400003EBEAFFEF500E6E0D6A0E500D5C15E2BA
:102F500009EBE9FF0AEBEAFF092A000E0A22EF500B
:102F6000E66E04EBE9FF05EBEAFF042A000E0522FA
:102F7000E552E750EF6E0D2AE8D7A4AE06D000EB7D
:102F8000E9FF01EBEAFFEF88A49E0BEBE9FF0CEBF6
:102F9000EAFFEF9E010E00D047E9E7CFD9FF12000C
:102FA000D9CFE6FFE1CFD9FF82E91F0E6F1600509F
:102FB0006F12E00E6E14005C01E0FBD741E9E7CF31
:102FC000D9FF1200D9CFE6FFE1CFD9FF88E942E867
:102FD000D950010FE66EDACFE6FFE552E550096EF3
:102FE000E750086E005034E108EBE9FF09EBEAFF17
:102FF000EF50E840E840E8401F0BE66E05EBE9FFC4
:1030000006EBEAFFE552E750EF6E08EBE9FF09EB4C
:10301000EAFFEE52EF50200DF3CFE0F005EBE9FFB1
:1030200006EBEAFF0001E051EF12052A000E06222E
:1030300008EBE9FF09EBEAFFEF50200DF350E66ED5
:1030400005EBE9FF06EBEAFFE552E750EF6E75D0BE
:1030500008EBE9FF09EBEAFF020EE926000EEA227F
:10306000EF50E00BE838E840E66E05EBE9FF06EBD1
:10307000EAFFE552E750EF6E08EBE9FF09EBEAFFE4
:10308000030EE926000EEA22EF50080DF3CFE0F020
:1030900005EBE9FF06EBEAFF0001E051EF12052A1C
:1030A000000E062208EBE9FF09EBEAFF020EE92613
:1030B000000EEA22EF50080DF350E00BE66E05EB30
:1030C000E9FF06EBEAFFE552E750EF6E05EBE9FF9B
:1030D00006EBEAFFEF8608EBE9FF09EBEAFF020ED9
:1030E000E926000EEA22EF50030BE06F05EBE9FF43
:1030F00006EBEAFFE051EF12052A000E062208EB6C
:10310000E9FF09EBEAFFEE52EF50E66E05EBE9FF4F
:1031100006EBEAFFE552E750EF6E052A000E0622A5
:1031200008EBE9FF09EBEAFFEF50E66E05EBE9FF7C
:1031300006EBEAFFE552E750EF6E43E9E7CFD9FF30
:103140001200D9CFE6FFE1CFD9FF86E942E881EB53
:1031500006F082EB07F0005046E103EBE9FF04EBD9
:10316000EAFFEF50080DF350E66E06EBE9FF07EBC0
:10317000EAFFE552E750EF6E03EBE9FF04EBEAFFED
:10318000EF50E00BE838E840E66E06EBE9FF07EBAE
:10319000EAFFEE52E552E750EF6E032A000E0422DA
:1031A00003EBE9FF04EBEAFFEF50E00BE838E840FF
:1031B0000001E06F06EBE9FF07EBEAFFE051EF12D9
:1031C00006EBE9FF07EBEAFF020EE926000EEA2212
:1031D000EF6A06EBE9FF07EBEAFF030EE926000EB4
:1031E000EA22EF6A73D003EBE9FF04EBEAFFEF504A
:1031F000200DF350E66E06EBE9FF07EBEAFF020E47
:10320000E926000EEA22E552E750EF6E03EBE9FFF4
:1032100004EBEAFFEF50E840E840E8401F0BE66EA1
:1032200006EBE9FF07EBEAFF030EE926000EEA22B0
:10323000E552E750EF6E032A000E042203EBE9FF8C
:1032400004EBEAFFEF50030B0001E06F06EBE9FF30
:1032500007EBEAFF020EE926000EEA22E051EF1228
:1032600003EBE9FF04EBEAFFEF50E00BE840E84036
:10327000E8401F0BE06F06EBE9FF07EBEAFF020EE9
:10328000E926000EEA22E051EF12032A000E042282
:1032900003EBE9FF04EBEAFFEF50E66E06EBE9FF14
:1032A00007EBEAFFEE52E552E750EF6E032A000EFD
:1032B000042203EBE9FF04EBEAFFEF50E66E06EBB6
:1032C000E9FF07EBEAFFE552E750EF6E43E9E7CF8E
:0432D000D9FF120010
:0C32D40043E8D9CFE6FFDACFE6FFE1CFF8
:1032E000D9FFE2CFDAFF89E9066A1200F3DF068030
:1032F00001D0F0DF01AE83EF19F0006C011EE86A27
:10330000012206B0067E03AE8BEF19F0026C031E9D
:10331000E86A0322067EC3EC19F003BEADEF19F094
:1033200006AE08D0026C031EE86A0322046C051E78
:10333000E86A052206B006D084EB00F085EB01F0C8
:1033400006A004D082EB00F083EB01F0E552E5CF5C
:10335000DAFFE7CFD9FF45E9000C06BE92EF19F07E
:10336000E9DFFF0C43E8D9CFE6FFDACFE6FFE1CF94
:10337000D9FFE2CFDAFF89E9066A1200F3DF06809F
:1033800003D0F0DF01D00682056A046A100EE76EF2
:10339000D89002360336043605360050045C0150DE
:1033A000055805E30050045E0150055A022AE72E35
:1033B000F0D706B2120006B006D084EB00F085EB21
:1033C00001F006A004D082EB00F083EB01F0E5529F
:1033D000E5CFDAFFE7CFD9FF45E9120045E8D9CFBD
:1033E000E6FFDACFE6FFE1CFD9FFE2CFDAFF8FE9E0
:1033F0000C6A1200F3DF0C8001D0F0DFE86A03AE44
:103400000BEF1AF0006C011E021E031E01220222A5
:1034100003220CB00C7E07AE16EF1AF0046C051EEA
:10342000061E071E0522062207220C7EE2EC1AF079
:1034300007BE47EF1AF00CAE0FD0046C051E061E37
:10344000071EE86A052206220722086C091E0A1ECA
:103450000B1E09220A220B220CB00AD088EB00F0C6
:1034600089EB01F08AEB02F08BEB03F00CA008D0A3
:1034700084EB00F085EB01F086EB02F087EB03F0C4
:10348000E552E5CFDAFFE7CFD9FF49E9000C0CBEE2
:103490001DEF1AF0E1DFFF0C44E8D9CFE6FFDACFE9
:1034A000E6FFE1CFD9FFE2CFDAFF8AE980EB04F053
:1034B00081EB05F082EB06F002500402F450016E3D
:1034C000F350006E0350076E0502F450036EF35084
:1034D000026E07500402F3500126F4500222E86AFB
:1034E000032206500502F3500126F4500222E86A36
:1034F0000322E552E5CFDAFFE7CFD9FF46E9000C1A
:1035000044E8D9CFE6FFDACFE6FFE1CFD9FFE2CF3B
:10351000DAFF8EE980EB08F081EB09F082EB0AF02C
:1035200083EB0BF004500802F350006EF450016E70
:1035300004500902F3500126000EF420026E0450DC
:103540000A02F3500226000EF420036E04500B0210
:10355000F350032605500802F3500126F4500222CE
:10356000000E032205500902F3500226F4500322F4
:1035700005500A02F350032606500802F3500226B3
:10358000F450032206500902F350032607500802A4
:10359000F3500326E552E5CFDAFFE7CFD9FF48E93C
:1035A000000C45E8D9CFE6FFDACFE6FFE1CFD9FF3F
:1035B000E2CFDAFF8FE90C6A1200F3DF0C8003D050
:1035C000F0DF01D00C820B6A0A6A096A086A200ED1
:1035D000E76ED890043605360636073608360936C3
:1035E0000A360B360050085C0150095802500A5840
:1035F00003500B5809E30050085E0150095A02506D
:103600000A5A03500B5A042AE72EE4D70CB21200D0
:103610000CB00AD088EB00F089EB01F08AEB02F0E5
:103620008BEB03F00CA008D084EB00F085EB01F0ED
:1036300086EB02F087EB03F0E552E5CFDAFFE7CF48
:06364000D9FF49E9120068
:0A364600DACFE4FFE2CFDAFFE9CFAC
:10365000E4FFEACFE4FFEEC0E4FFEFC0E4FFF0C018
:10366000E4FFF1C0E4FFF6CFE4FFF7CFE4FFF5CFCE
:10367000E4FFF3CFE4FFF4CFE4FFFACFE4FF00EE82
:10368000E0F0080EE80403E3EECFE4FFFBD7E652D8
:10369000D9CFE6FFE1CFD9FF81E941E8A4BCA49CE2
:1036A000F2A46FD0F294CB0ED66EF30ED76E00015B
:1036B000DF2B640EE76EDF1902E7E73402D0E75034
:1036C000DF5D03E3DF6B829008D05F0EDF5D05E115
:1036D000040E0001A05D01E082800001DA2B050EDE
:1036E000E76EDA1902E7E73402D0E750DA5D33E338
:1036F000DA6B0001AD5101E0AD070001D95101E0E5
:10370000D907D751D81103E0D707000ED85BDB519A
:1037100001E0DB078150016E300E0114300801E139
:10372000DD6B3C0EE76EDD1902E7E73402D0E750AF
:10373000DD5D0DE20150DC15100B02E07AEC10F0BB
:1037400001500001DC15200B02E08CEC10F0011C94
:103750000001DC6FDD2BDE2B0A0EE76EDE1902E7BF
:10376000E73402D0E750DE5D0CE3C2B208D0FF0EB2
:10377000C3140001B06F030EC414B16FC282000104
:10378000DE6B42E9E7CFD9FFE55200EEE7F0080E25
:10379000E80403E3E5CFEDFFFBD7E5CFFAFFE5CF84
:1037A000F4FFE5CFF3FFE5CFF5FFE5CFF7FFE5CF7A
:1037B000F6FFE5CFF1F0E5CFF0F0E5CFEFF0E5CFA4
:1037C000EEF0E5CFEAFFE5CFE9FFE5CFDAFF110044
:1037D0008A6A8B6A92689368B80E946E040ED56EEE
:1037E000CB0ED66EF30ED76ED58EF19E010EC26E45
:1037F0000E0EC16EBE0EC06EC282600EF26EF28EF2
:023800001200B4
:0E3802000E0EF66E000EF76E000EF86E000150
:103810000900F550D26F0900F550D36F03E1D2676C
:1038200001D03DD00900F550CD6F0900F550CE6FA5
:103830000900F550CF6F09000900F550E96E090045
:10384000F550EA6E090009000900F550D06F090033
:10385000F550D16F09000900F6CFD4F0F7CFD5F0BD
:10386000F8CFD6F0CDC0F6FFCEC0F7FFCFC0F8FF3F
:103870000001D05302E1D15307E00900F550EE6E8C
:10388000D007F8E2D107F9D7D4C0F6FFD5C0F7FFCB
:10389000D6C0F8FF0001D207000ED35BBFD71200DD
:1038A000D9CFE6FFDACFE6FFE1CFD9FFE2CFDAFFEB
:1038B00087E944E8D9CFE6FFDACFE6FFE552E550E5
:1038C0000A6EE750096E09EBE6FF0AEBE6FF00EB34
:1038D000E6FF01EBE6FF02EBE6FFD950030FE66ED1
:1038E000000EDA20E66EC1EC11F047E9F350076EE6
:1038F000F450086E03EBE9FF04EBEAFFEF6A07EB15
:10390000F3FF08EBF4FF45E9E5CFDAFFE7CFD9FF96
:023910001200A3
:0E391200FE0EE3CFE9FFFF0EE3CFEAFFF36AFC
:10392000F46AEE5203E0F34AF42AFBD71200FF0ECA
:10393000E3CFF8FFE552FF0EE3CFF7FFE552FF0EAE
:10394000E3CFF6FFE552E66AE66AE66A0900F55259
:1039500009E0FD0EE32A05E1FE0EE32A02E1FF0E77
:10396000E32AF4D7FD0EE3CFEEF0FE0EE3CFEFF047
:08397000FF0EE3CFF0F012009E
:08397800D9CFE6FFDACFE6FF2C
:10398000E1CFD9FFE2CFDAFF85E9013415E200EBA0
:10399000E9FF01EBEAFFEECFF3FFEDCFF4FFEE2AF4
:1039A000000EEF22F3CFE9FFF4CFEAFF02EBEFFFC7
:1039B000EF50F36EF46A0DD0FE0E005C05E102EBF1
:1039C000E6FF3DEC1DF004D002EBE6FF03EC00F057
:0E39D00041E941E9E5CFDAFFE7CFD9FF120068
:0239DE004E6F2A
:1039E0002043414E2D425553205369676E616C73DD
:1039F0002E0056312E303200556E7265636F676E41
:103A0000697A65642053442E004E6F204249544D1C
:103A1000415020534420434152442E00253264003B
:103A20002D302D312D322D332D342D352D362D3792
:053A30000049443A00CA
:0A3A3600F36AF46AFF0EE124E96E62
:103A4000FF0EE220EA6EED6607D02F0EEF6404D081
:0A3A50003A0EEF6001D0F32A1200D5
:063A5A00000EF36E00EE09
:103A600000F00D0E01D81200EA6002D0EE6AFCD719
:0A3A7000F350E9601200EE6AFCD783
:063A7A00FF0EE350ACBAA0
:103A800004D0AF6AAB8EAC8A949CACA2FED7AD6E6C
:063A9000F36EF46A12005F
:0A3A96001CEE00F02CEE00F0F86AC0
:103AA00001EC1CF061EC1DF0A4EC0AF0FBD7120055
:103AB00030313233343536373839616263646566A4
:013AC0000005
:023AC2001200F0
:093AC400000000000000000000F9
:020000040030CA
:0100010006F8
:0100020000FD
:010003001EDE
:01000500807A
:01000600C138
:00000001FF
